:020000040000fa
:0800000082050400000000006d
:020000040000fa
:020000040002f8
:04afe000dfff00008f
:020000040000fa
:020000040002f8
:04afe400ffff00006b
:020000040000fa
:020000040002f8
:04afe80078ff0000ee
:020000040000fa
:020000040002f8
:04afec007dff0000e5
:020000040000fa
:020000040002f8
:04aff00078ff0000e6
:020000040000fa
:1000080000000000000000000000000000000000e8
:100018007a05000000000000000000000000000059
:10002800e209000000000000000000006e0a000065
:1000380000000000000000000000000000000000b8
:100048009e0a000000000000000000006e0b000087
:10005800da0b00000a0c000000000000000000009d
:100068000000000000000000000000000000000088
:100078000000000000000000000000000000000078
:10008800000000000000000000000000ca0a000094
:100098003e0b00000000000000000000000000000f
:1000a8000000000000000000000000000000000048
:1000b8000000000000000000000000000000000038
:1000c8000000000000000000000000000000000028
:1000d8000000000000000000000000000000000018
:1000e8000000000000000000000000000000000008
:1000f80000000000000000000000000000000000f8
:1001080000000000000000000000000000000000e7
:1001180000000000000000000000000000000000d7
:1001280000000000a60b0000000000000000000016
:1001380000000000000000000000000000000000b7
:1001480000000000000000000000000000000000a7
:100158000000000000000000000000000000000097
:100168000000000000000000000000000000000087
:100178000000000000000000000000000000000077
:100188000000000000000000000000000000000067
:100198000000000000000000720c00009e0c00002f
:1001a800ca0c000000000000000000000000000071
:1001b8000000000000000000000000000000000037
:1001c8000000000000000000000000000000000027
:1001d8000000000000000000000000000000000017
:1001e8000000000000000000000000000000000007
:1001f80000000000000000000000000000000000f7
:1002080000000000000000000000000000000000e6
:1002180000000000000000000000000000000000d6
:1002280000000000000000000000000000000000c6
:1002380000000000000000000000000000000000b6
:1002480000000000000000000000000000000000a6
:100258000000000000000000000000000000000096
:100268000000000000000000000000000000000086
:0c0278000000000000000000000000007a
:020000040000fa
:10040000803e2000030007008100e900fcff3a0065
:1004100000000600831f7800c20320000400bc0017
:1004200066015100e0815900f23fb1000380b10044
:1004300006003500ee03090000000000423fb10055
:100440000380b100fbff3d001200b000223fb0006e
:10045000020035000280090000000000cf01780092
:1004600000000600861f78006022b8000602200007
:100470000000d0008180d2000482d2008582d200a8
:100480000000a0000202520083825a0003003100e3
:100490000202420083824a000000a1000603e90034
:1004a000f3ff3a004f03780000000600889fbe006b
:1004b0008a9fbe008c1f78000004be004101070027
:1004c0000478a30026003a006120e10025003200f4
:1004d00009f8a30025003a006420e1002100320061
:1004e000f507b1000508a30002003200000040003b
:1004f000818048006044b800031020000200200002
:1005000000004000818048000805440089854c00b7
:100510000a0541008b8549000a0550008b8558006b
:10052000030033000a00be000204740083847400d8
:100530008301d1000281d300830f7100f0ff3a00e4
:100540008904d1000884d300600149008201780049
:10055000c1adde00fb07b0002f0107000700370028
:100560000960a0000800be0004003700120220004d
:1005700062928800f0ff2f00f1ff27004f067800fd
:100580004f05be004f04be000000060003f0a200ad
:10059000869fbe00889fbe008a9fbe008c9fbe00c3
:1005a00000010700420133006450e1004f003200b7
:1005b0006420e1005200320003826c0007003b001f
:1005c0000905d0000306d000820f54000c065d0020
:1005d0000200390002003200890178000306780029
:1005e0008582550004003d000003fd008103fd00ed
:1005f0008502ea008b854200840f720002003b00f6
:1006000060001000e08018006011b8000005eb00e9
:100610007a28e1000a00390006007800c75ddd0095
:10062000f707b200878075002d00370082817100c6
:100630000a017800610560008180d1000080d3004c
:100640008502e900f9ff3b0006044000878448006a
:1006500002003b0060041400e0841c000988a30031
:10066000070032008a81710082817100610164009b
:100670008904d1000884d3008b05e80017003700f7
:100680000978a30013003a000b00e00013003400c7
:100690008b05e9000804440089844c000a44740076
:1006a0000978a3000d003a000b00e00007003400b9
:1006b0008b05e9000804440089844c0001003a00dd
:1006c0000b0020000978a300f7ff32000001eb00c7
:1006d00002003700828171000a017800ce00070015
:1006e0000cf0a70001f0a000fa0037006420e10040
:1006f00002003a00838f6c00fb0033000801be004b
:100700000200be00f3003700869fbe00889fbe0037
:100710008a9fbe008c9fbe00a2000700e400330049
:1007200003866c006450e100240032006420e10084
:10073000270032006150e100220032006120e10018
:10074000210032008b854200eb07b1000134b80074
:10075000003ab8000804420089844a00013ab8000f
:100760000030b8008880400009014a0004003300ce
:100770000000400081804800020149008b05e9002b
:10078000c909dd0083017000010032001300200060
:10079000c814de004814dd004709de001200b20074
:1007a000c808de00088470009b00070001f0a1006b
:1007b0000cf0a70001f0a000c60037006120e100a6
:1007c000c90032000801be000200be00f7ff37007a
:1007d0006150e100fcff3a00c3003700829fbe0079
:1007e0000001be00770007000470a70003f0a1001d
:1007f0006509b100180032000e0035006828e100dc
:1008000007003500f0ff2f00f1ff27000300e00094
:1008100015003b00010028004f01be00000005004c
:1008200000004000818048008502e900fcff3a009a
:1008300009003700f88f420003003c008000eb0005
:100840004f01be00000005008100d1000080d300f0
:100850008502e800fcff3a000300e00002003b00d4
:1008600060001000e08018004f01be00000006008c
:10087000829fbe000001be00520007000470a70066
:1008800003f0a10003f8a30015003a006509b100c8
:10089000110032000a0035006928e100030035002c
:1008a000010028004f01be000000050000004000cc
:1008b000818048008502e900fcff3a00060037000d
:1008c000f88f4200060035008100d1000080d3007f
:1008d0008502e800fcff3a004f01be000000060060
:1008e0008000eb004f01be00000005008000eb001f
:1008f000829fbe00889fbe008a9fbe0001057800cf
:100900000100e0000400350008003c000000e000a9
:10091000200032000500370060001000e080180061
:1009200002003b0001f024001a0037000004be0062
:100930006011b8006b0920000982cf000200390065
:100940000882cf000441b000694252000e0032001c
:1009500008003b0082817100610164008904d100bc
:100960000884d3008b05e8000442e800f9ff3a0050
:10097000050037000804440089844c008b05e90019
:100980000442e900fbff3a00230007000af0a70039
:1009900001f0a0004f05be004f04be004f01be0095
:1009a000000006000004be00060007000003be00b1
:1009b0000405be000200be0002000700844f75005f
:1009c00000000600c70ade00f107b200f50fb20012
:1009d00008003200e1cf4200020032000170a000a6
:1009e00024000500810f700001003200040805009a
:1009f00044000500810f700002003a001400050059
:100a00008502e9000000400081c04800fcff3b0077
:100a10000170a000240005008100200061805500c5
:100a20000b003d000b00200061fe2f000100e100e3
:100a30001d00340082817100610164008904d100cd
:100a40000884d3000000e800faff3a00710020009b
:100a500061006400030070000200600009003200c1
:100a600061044400e0844c000988a50005003200c0
:100a70008b05e8006808e10002003a008904d10013
:100a80000884d300f20f20000258e10005003d0069
:100a9000c75ddd00f907b2008980750008007800a5
:100aa000000006000bf827008b007800000005000e
:100ab0000200be006450e100050036006420e10041
:100ac000020036000968a30001003a000800be00d9
:100ad0000160a0004f06be004f05be004f04be00df
:100ae0004f03be0000000600f0ff2f00f1ff2700bb
:100af000f8ff37000020ef000220ef00c088a900b7
:100b0000004006000f002100403221000001880053
:100b1000000000000000eb00000778000c00090056
:100b2000002f78000007eb005420ef000e2eef009e
:100b30001e2eef000000eb0001242100bf1d090064
:100b40008018780040a7a900a10020002cfe070013
:100b5000e0022000303a880044e7a90044c7a90019
:100b60004407a9004427a9004447a9004467a900f5
:100b70004487a900300020000600fc0031742000ea
:100b800082072000a309200082487800834878006b
:100b900080487800113a8000618070000600fc00f7
:100ba0002174200062042000730520008248780030
:100bb00083487800804878004427ef00e002200056
:100bc000303a8800300020000d00fc003174200015
:100bd00082072000a309200082487800834878001b
:100be000804878000000200021742000620420006a
:100bf0007305200082487800834878008048780098
:100c000042a7ae00feff3700813e2000fcfd07003a
:100c100010c0b30086e6b70090c2b300c4e6b700c8
:100c2000000ea800007825008070880010cea90072
:100c3000108ea90010aea900008ea9004188a8005e
:100c400041a8a90041c8a90004a1a8000481a800e6
:100c500005e1a8000068a9000021ef0002a1ef0053
:100c60002068a8001061a8001021a90011e1a800c7
:100c700011a1a90010a1a8001081a8000621ef0071
:100c80000a21ef000ca1ef000ea1ef004408a9001b
:100c90004428a9004448a9000108a9002108a80087
:100ca0001fe1a8001fa1a9001ec1a9001ea1a80044
:100cb0001e81a8001e61a9001e21a9004d88a80060
:100cc0004da8a8004dc8a900803e2000d00888008b
:100cd0000368a9002368a80021e1a80021a1a900b8
:100ce00020c1a90020a1a8002081a8002021a900de
:100cf0004e08a8004e28a9004e48a8000388a90065
:100d0000a00e2000e00888002388a8002002a90087
:100d10002022a9002042a90020a2a9002062a90047
:100d20002082a90020e2a9002102a9002122a90015
:100d3000700720004011880022a2a90022c2a90049
:100d400022e2a90021e2a8002182a9004588a90089
:100d500045a8a80045c8a8002168a8002828a80020
:100d600023e2a9002342a8002362a9000188a90068
:100d70002188a8004608a9004628a8004648a800df
:100d80000e0ea80021e3a9002143a80021a3a90079
:100d90002123a9002103a90020e3a90020c3a90061
:100da00020a3a9002083a9002043a80023e3a900d1
:100db00023c3a90023a3a9002343a9002323a90037
:100dc0002303a90022c3a90022a3a9002283a9000a
:100dd0002263a9002243a9002223a9002203a9001b
:100de0002563ef0024e3ef003223ef002823ef0018
:100df0002623ef002e23ef003023ef0021a8a800c8
:100e000046c8a80046a8a9004688a80001a8a900cd
:100e100021e3a8004008a9004028a9004048a800f4
:100e20002008a8000008a900c208a80080c0b300dc
:100e3000c8e8b7002bc8a9002be8a9002c08a90016
:100e40000bc8a9000be8a9000c08a90001eca90037
:100e500001aca900016ca900014ca900012ca9005a
:100e6000010ca90000eca900008ca90000aca900ad
:100e700000cca900000ca900002ca900004ca9007e
:100e8000006ca900202cef00402cef00602cef003c
:100e90000000210020608800020ca900022ca9009b
:100ea000024ca900262cef00462cef00662cef0028
:100eb000282cef00482cef00682cef000aacef0064
:100ec00023eca80023cca80023aca900238ca90004
:100ed000236ca900234ca800232ca900230ca900f3
:100ee000222ca80043eca80043cca80043aca900e6
:100ef000438ca900436ca800434ca900432ca900d3
:100f0000430ca90063eca80063cca80063aca90063
:100f1000638ca800636ca800634ca900dabc2a00ab
:100f20001b32240030002c00fa608800fb6088002f
:100f300020618800dabc2a001b32240020402c00eb
:100f4000fa608800fb60880010618800dabc2a0023
:100f50001b32240030002c00fa608800fb608800ff
:100f600020628800dabc2a001b32240000802c009a
:100f7000fa608800fb60880010628800dabc2a00f2
:100f80001b32240030002c00fa608800fb608800cf
:100f900020638800dabc2a001b32240000802c0069
:100fa000fa608800fb60880010638800a7003700a3
:100fb0003f00370000202000006188000020200052
:100fc000006288000020200000638800020ca90055
:100fd000022ca800024ca80004acef0028acef00e3
:100fe00048acef0068acef00262cef00462cef0079
:100ff000662cef000aacef0023eca80023cca9007c
:1010000043eca80043cca90063eca80063cca90082
:10101000dabc2a001b32240030002c00fa60880061
:10102000fb60880020618800dabc2a001b322400a3
:1010300000002800fa608800fb60880010618800ca
:10104000dabc2a001b32240030002c00fa60880031
:10105000fb60880020628800dabc2a001b32240072
:1010600000002800fa608800fb6088001062880099
:10107000dabc2a001b32240030002c00fa60880001
:10108000fb60880020638800dabc2a001b32240041
:1010900000002800fa608800fb6088001063880068
:1010a00011eea90011aea900116ea900670037006a
:1010b000350037000010200000618800001020007b
:1010c000006288000010200000638800020ca90064
:1010d000022ca800024ca8000a2cef0004acef0080
:1010e000282cef005055250040628800a0aa2a0055
:1010f00040638800dabc2a001b32240030002c0038
:10110000fa608800fb60880020618800dabc2a0051
:101110001b32240000002c00fa608800fb6088006d
:1011200010618800dabc2a001b32240030002c0039
:10113000fa608800fb60880020628800dabc2a0020
:101140001b32240000002c00fa608800fb6088003d
:1011500010628800dabc2a001b32240030002c0008
:10116000fa608800fb60880020638800dabc2a00ef
:101170001b32240000002c00fa608800fb6088000d
:101180001063880031003700300037000010200065
:10119000006188000010200000628800020ca90095
:1011a000022ca800024ca8000a2cef0004acef00af
:1011b000282cef000000240040628800dabc2a00de
:1011c0001b32240030002c00fa608800fb6088008d
:1011d00020618800dabc2a001b32240000002c00a9
:1011e000fa608800fb60880010618800dabc2a0081
:1011f0001b32240030002c00fa608800fb6088005d
:1012000020628800dabc2a001b32240000002c0077
:10121000fa608800fb60880010628800dabc2a004f
:101220001b32240030002c00fa608800fb6088002c
:1012300020638800dabc2a001b32240000002c0046
:10124000fa608800fb60880010638800218ca90088
:10125000418ca900618ca900216ca900416ca900f6
:10126000616ca900214ca900414ca900614ca90066
:1012700020eca80040eca80060eca8003e2cef0099
:101280005e2cef007e2cef0001eca80080b2ef0096
:101290000000eb00a19d2100ff00090080587800ac
:1012a000a772ef00a872ef009632ef009832ef00bd
:1012b0000000eb00a1ad2100ff000900805878007c
:1012c000a972ef00aa72ef000080eb00619c210080
:1012d00009000900801878000000eb00612c210053
:1012e000ff00090080187800bb72ef00bc72ef00ad
:1012f0000000eb00614c2100ff000900801878001d
:10130000bd72ef000000eb00616c2100ff000900de
:1013100080187800be72ef00bf72ef00108ea90037
:10132000148ea900008ea900048ea90010aea90099
:1013300014aea9002008a8002068a80021a8a800d1
:1013400001a8a900262cef002003a9002023a80053
:1013500000122000e00888000388a9002388a80064
:10136000803e2000d00888000368a9002368a800f8
:1013700000802000809388007e32ef007c32ef00f6
:101380007a32ef009432ef009032ef009232ef00a9
:1013900000c4b30082f2b70000c4b30084f2b70007
:1013a000a0c0b30088f2b70040002000509488002d
:1013b00060002000609488003f0707003e08070097
:1013c00097013700ff3ffc004200f8003600f800ac
:1013d0004400f8008e1f78000e0020000d00090068
:1013e000be1f78003200f8004012f8004212f800e8
:1013f0000100fc000008a9006612ae000c003700d6
:101400000021ef006612a9006a32ef00be72ec0004
:10141000bed2bf000080fb000000d000616c210044
:101420000100400001002000010878001e00370084
:101430000008800040938800509380000100200045
:10144000f21f2000030020000001410081814900bb
:101450004093800001002000820f5000838f5800cd
:101460000f0036000021ef006a32ef00be72ec0080
:1014700042938000030020000000200011002000a3
:10148000f8fb0700e12b2100914078008180fb00f0
:1014900081804000626c21008030790002003700ba
:1014a0004093800050938800ff3ffc004212f900f7
:1014b0004012f9003200f900ae0120000d000900d1
:1014c0004f1778004f0778004400f9003600f90004
:1014d0004200f9000100fc0000400600ff3ffc0054
:1014e0004200f8003600f8004400f8008e1f780033
:1014f0000e0020000d000900be1f78003200f80029
:101500000100fc000068a9000021ef006612a8009d
:10151000ff3ffc003200f900ae0120000d00090081
:101520004f1778004f0778004400f9003600f900a3
:101530004200f9000100fc0000400600ff3ffc00f3
:101540004200f8003600f8004400f8008e1f7800d2
:101550000e0020000d000900be1f78003200f800c8
:101560000100fc000108a900ff3ffc003200f90067
:10157000ae0120000d0009004f1778004f077800da
:101580004400f9003600f9004200f9000100fc00b7
:1015900000400600ff3ffc004200f8003600f80063
:1015a0004400f8008e1f78000e0020000d00090096
:1015b000be1f78003200f8004012f8000100fc0065
:1015c0000368a9001421ef006c32ef005232ef00e3
:1015d000bed2bf00bf52e3000a003200bf72ec006f
:1015e0005232ec00bfd2bf000080fb000000400080
:1015f000616c2100608078006c12b40060938800f8
:10160000f3ff37005212e2000700360060938000bb
:10161000929280000200e0000200320011000900f6
:101620000280d80060938800800c20000100200018
:10163000b2948000c394800002014000838148007e
:10164000b2ce8800c3ce8800ba12a800ff3ffc00cb
:101650004012f9003200f900ae0120000d0009002f
:101660004f1778004f0778004400f9003600f90062
:101670004200f9000100fc0000400600ff3ffc00b2
:101680004200f8003600f8004400f8008e1f780091
:101690000e0020000d000900be1f78003200f80087
:1016a0000100fc000388a9001821ef002023a900f5
:1016b000ff3ffc003200f900ae0120000d000900e0
:1016c0004f1778004f0778004400f9003600f90002
:1016d0004200f9000100fc0000400600ff3ffc0052
:1016e0004200f8003600f8004400f8008e1f780031
:1016f0000e0020000d000900be1f78003200f80027
:101700000100fc000168a900a772ec00a7d2bf008d
:101710008080fb0030118000a29d21008070790044
:10172000ff3ffc003200f900ae0120000d0009006f
:101730004f1778004f0778004400f9003600f90091
:101740004200f9000100fc0000400600ff3ffc00e1
:101750004200f8003600f8004400f8008e1f7800c0
:101760000e0020000d000900be1f78003200f800b6
:101770000100fc000828a9002242ae00000037004a
:101780002222af002222a900ff3ffc003200f90014
:10179000ae0120000d0009004f1778004f077800b8
:1017a0004400f9003600f9004200f9000100fc0095
:1017b00000400600ff3ffc004200f8003600f80041
:1017c0004400f8008e1f78000e0020000d00090074
:1017d000be1f78003200f8000100fc000188a9005b
:1017e000128eaa00108ea900ff3ffc003200f90003
:1017f000ae0120000d0009004f1778004f07780058
:101800004400f9003600f9004200f9000100fc0034
:1018100000400600ff3ffc004200f8003600f800e0
:101820004400f8008e1f78000e0020000d00090013
:10183000be1f78003200f8000100fc0001a8a900da
:101840002003a90000188000709388008093800016
:1018500071938000808f50000400360080938000d8
:101860006e12b500c09388000300370070938000ab
:101870007012b500c0938800b09380007812b40055
:10188000a0938800c0938000b0938800709380007c
:10189000809388008007200001002000b29480001f
:1018a000c3948000020140008381480092ce8800ea
:1018b000a3ce8800ba12a800ff3ffc003200f90056
:1018c000ae0120000d0009004f1778004f07780087
:1018d0004400f9003600f9004200f9000100fc0064
:1018e00000400600ff3ffc004200f8003600f80010
:1018f0004400f8008e1f78000e0020000d00090043
:10190000be1f78003200f8000100fc000bc8a900df
:10191000ff3ffc003200f900ae0120000d0009007d
:101920004f1778004f0778004400f9003600f9009f
:101930004200f9000100fc0000400600ff3ffc00ef
:101940004200f8003600f8004400f8008e1f7800ce
:101950000e0020000d000900be1f78003200f800c4
:101960000100fc000be8a900ff3ffc003200f90079
:10197000ae0120000d0009004f1778004f077800d6
:101980004400f9003600f9004200f9000100fc00b3
:1019900000400600ff3ffc004200f8003600f8005f
:1019a0004400f8008e1f78000e0020000d00090092
:1019b000be1f78003200f8000100fc000c08a900ee
:1019c000ff3ffc003200f900ae0120000d000900cd
:1019d0004f1778004f0778004400f9003600f900ef
:1019e0004200f9000100fc0000400600a8d2bf0040
:1019f000a752e30007003200a872ec00a8d2bf0093
:101a00000080fb00a19d210060c07800abf2b70010
:101a100001003700abf2ef000000060000000600f6
:101a200001948000e18f50000d003a00a972ec0093
:101a3000a9d2bf000080fb00720d2000a1ad2100e3
:101a400002f07800a972ec00a9d2bf000080fb0070
:101a500012002000a1ad210002f078008032ef00da
:101a600050088000c094880030088000b09488003e
:101a7000deff070080ceb300ab52b5000600390090
:101a8000e0cfb300ab52b5000100390001003700d0
:101a9000ac72ef007a013700abf2ae0037003700ce
:101aa000ac72ef0070c8b300ab52e30005003a001f
:101ab000abd2bf00acf2b700adf2ef00aef2ef0078
:101ac0002d00370070c9b300ab52e30005003a00a7
:101ad000abd2bf00acf2b700aff2ef00b0f2ef0054
:101ae0002500370070cab300ab52e30005003a008e
:101af000abd2bf00acf2b700b1f2ef00b2f2ef0030
:101b00001d00370070cbb300ab52e30005003a0074
:101b1000abd2bf00acf2b700b3f2ef00b4f2ef000b
:101b20001500370070ccb300ab52e30004003a005c
:101b3000abd2bf00acf2b700b5f2ef000e00370039
:101b400070cdb300ab52e30004003a00abd2bf004b
:101b5000acf2b700b6f2ef000700370070ceb3006a
:101b6000ab52e30004003a00abd2bf00acf2b700c6
:101b7000b7f2ef00b8f2ef0041013700ac52e200db
:101b800002003a003e0137003d01370070c8b30043
:101b9000ac52e3003d003a0000e0ef00ad52e3003c
:101ba00003003a00abd2bf00adf2b70036003700f9
:101bb000abd2bf00aef2b700add2bf00f1c2b300ee
:101bc00080cf100016003600e0c4b300ad52e30031
:101bd00013003e00a972ec00a9d2bf000080fb00f8
:101be00072082000a1ad210002f07800a972ec007b
:101bf000a9d2bf000081fb00a1ad2100add2bf0082
:101c000000f17800a972ec00a9d2bf000081fb00ae
:101c1000a1ad2100aed2bf0000f17800190037005d
:101c2000add2bf00f1c6b30080cf10001500360062
:101c3000f0c7b300ad52e30012003e00a972ec0001
:101c4000a9d2bf000080fb0072082000a1ad2100d6
:101c500002f07800a972ec00a9d2bf000081fb005d
:101c6000a1ad2100add2bf0000f17800a972ec0057
:101c7000a9d2bf000081fb00a1ad2100aed2bf0000
:101c800000f17800adf2ef00fd00370070c9b3003d
:101c9000ac52e30073003a0000e0ef00af52e30003
:101ca00003003a00abd2bf00aff2b7006c003700c0
:101cb000abd2bf00b0f2b700b052e20034003a003d
:101cc000afd2bf00f1c2b30080cf100016003600c3
:101cd000e0c4b300af52e30013003e00a972ec0071
:101ce000a9d2bf000080fb0072092000a1ad210035
:101cf00002f07800a972ec00a9d2bf000081fb00bd
:101d0000a1ad2100afd2bf0000f17800a972ec00b4
:101d1000a9d2bf000080fb0002002000a1ad21007d
:101d200002f0780019003700afd2bf00f1c6b3004f
:101d300080cf100015003600f0c7b300af52e300ab
:101d400012003e00a972ec00a9d2bf000080fb0087
:101d500072092000a1ad210002f07800a972ec0008
:101d6000a9d2bf000081fb00a1ad2100afd2bf000e
:101d700000f17800a972ec00a9d2bf000080fb003e
:101d800002002000a1ad210002f0780033003700ee
:101d9000afd2bf00f1c2b30080cf100016003600f2
:101da000e0c4b300af52e30013003e00a972ec00a0
:101db000a9d2bf000080fb0072092000a1ad210064
:101dc00002f07800a972ec00a9d2bf000081fb00ec
:101dd000a1ad2100afd2bf0000f17800a972ec00e4
:101de000a9d2bf000081fb00a1ad2100b0d2bf008d
:101df00000f1780019003700afd2bf00f1c6b30080
:101e000080cf100015003600f0c7b300af52e300da
:101e100012003e00a972ec00a9d2bf000080fb00b6
:101e200072092000a1ad210002f07800a972ec0037
:101e3000a9d2bf000081fb00a1ad2100afd2bf003d
:101e400000f17800a972ec00a9d2bf000081fb006c
:101e5000a1ad2100b0d2bf0000f17800aff2ef00d9
:101e60008700370070cab300ac52e30023003a0089
:101e700000e0ef00b152e30003003a00abd2bf0034
:101e8000b1f2b7001c003700abd2bf00b2f2b7000e
:101e9000b1d2bf00f1c2b30080cf100015003600f0
:101ea00010c6b300b152e30012003e00a972ec006c
:101eb000a9d2bf000080fb00720a2000a1ad210062
:101ec00002f07800a972ec00a9d2bf000081fb00eb
:101ed000a1ad2100b1d2bf0000f17800a972ec00e1
:101ee000a9d2bf000081fb00a1ad2100b2d2bf008a
:101ef00000f17800b1f2ef006100370070cbb30061
:101f0000ac52e3000a003a0000e0ef00b352e300f5
:101f100003003a00abd2bf00b3f2b70003003700b2
:101f2000abd2bf00b4f2b700f30207005400370091
:101f300070ccb300ac52e30029003a0000e0ef009f
:101f4000b552e30025003a00abd2bf00b5f2b700ae
:101f5000b552e2000d003a00a972ec00a9d2bf0010
:101f60000080fb00720c2000a1ad210002f078007f
:101f7000a972ec00a9d2bf000081fb00a1ad210035
:101f8000b5d2bf0000f1780013003700b5d2bf0012
:101f9000b1c0b30080cf10000f00360070c1b30095
:101fa000b552e3000c003e00a972ec00a9d2bf00bc
:101fb0000080fb00720c2000a1ad210002f078002f
:101fc000a972ec00a9d2bf000081fb00a1ad2100e5
:101fd000b5d2bf0000f17800b5f2ef00280037005d
:101fe00070cdb300ac52e30007003a0000e0ef0010
:101ff000b652e30003003a00abd2bf00b6f2b7001e
:10200000b6f2ef001e00370070ceb300ac52e30012
:102010001b003a0000e0ef00b752e30003003a0073
:10202000abd2bf00b7f2b70015003700abd2bf008c
:10203000b8f2b700a972ec00a9d2bf000080fb0083
:10204000720e2000a1ad210002f07800a972ec0010
:10205000a9d2bf000081fb00a1ad2100b7d2bf0013
:1020600000f17800a972ec00a9d2bf000081fb004a
:10207000a1ad2100b8d2bf0000f17800b7f2ef00a7
:102080007c12e20078013a007e12e20001003a0080
:1020900007040700010020009832af001140b00093
:1020a0009212af001140b100940032009212a800c9
:1020b0009832ae009212a900bdd2bf000080fb0092
:1020c00000004000614c2100608078005294800044
:1020d0000200e00002003200110009000280d80076
:1020e0007094880071948000ef8f500002003600d9
:1020f000f00020007094880072948000a0bd210040
:1021000060407900c0f2b700bbd2bf000080fb0086
:1021100000004000612c210060c07800c4f2b700cc
:1021200088d2bf00c452e3002e003600a972ec0032
:10213000a9d2bf000080fb0072092000a1ad2100e0
:1021400002f07800a972ec00a9d2bf000081fb0068
:10215000a1ad2100c0d2bf0000f17800a972ec004f
:10216000a9d2bf000081fb00a1ad2100c4d2bf00f5
:1021700000f17800c0d2bf00c1f2b700d093800058
:102180008c12bc00a294880090fd2f00a0948800bf
:10219000a194800070052000808f50000200340060
:1021a00070052000a0948800800220009412b400e2
:1021b000000678000c064600608c210060007e005e
:1021c000b2948000c394800000004100e080490088
:1021d0000001be0032ce880043ce8800ba12a800ab
:1021e00018003700c152e20016003600a972ec0058
:1021f000a9d2bf000080fb0072082000a1ad210021
:1022000002f07800a972ec00a9d2bf000081fb00a7
:10221000a1ad2100c1d2bf0000f17800a972ec008d
:10222000a9d2bf000080fb0002002000a1ad210068
:1022300002f07800c172ef00c6b9ef00c8b9ef0034
:10224000ba12a8006612ae00160037009052af0016
:1022500013003700a972ec00a9d2bf000080fb0078
:1022600072092000a1ad210002f07800a972ec00f3
:10227000a9d2bf000080fb0032072000a1ad2100e1
:1022800002f07800a972ec00a9d2bf000080fb0028
:10229000f2072000a1ad210002f078009052a800c2
:1022a000150037009052ae0013003700a972ec0001
:1022b000a9d2bf000080fb0072082000a1ad210060
:1022c00002f07800a972ec00a9d2bf000080fb00e8
:1022d00032072000a1ad210002f07800a972ec00c5
:1022e000a9d2bf000080fb0002002000a1ad2100a8
:1022f00002f078009052a900aa00370001002000e7
:102300009872af001140b0009232af001140b1009e
:10231000690032009232a8009872ae009232a90091
:10232000bdd2bf000080fb0000004000614c2100d6
:102330006080780062002000110009000280d8004f
:102340007094880071948000f58f50000200360070
:10235000500120007094880072948000a0be21007b
:1023600060407900c2f2b700bbd2bf000080fb0022
:1023700000004000612c210060c07800c4f2b7006a
:1023800088d2bf00c452e30029003600c3d2bf0088
:10239000c252e30025003200c472d500c472d500d9
:1023a000a972ec00a9d2bf000080fb00720a2000d5
:1023b000a1ad210002f07800a972ec00a9d2bf0003
:1023c0000081fb00a1ad2100c2d2bf0000f1780066
:1023d000a972ec00c4d2bf000080fb00f005b00081
:1023e000912a2100914078008180fb00a2ad21005c
:1023f00080707900c2d2bf00c3f2b700a972ec00ae
:10240000a9d2bf000080fb00720d2000a1ad210009
:1024100002f07800a972ec00a9d2bf000081fb0095
:10242000a1ad2100c2d2bf0000f178002100370029
:10243000c352e2001f003600a972ec00a9d2bf000f
:102440000080fb00720a2000a1ad210002f078009c
:10245000a972ec00a9d2bf000081fb00a1ad210050
:10246000c3d2bf0000f17800a972ec00a9d2bf006e
:102470000080fb0002002000a1ad210002f07800e6
:10248000c372ef00a972ec00a9d2bf000080fb006c
:10249000720d2000a1ad210002f07800a972ec00bd
:1024a000a9d2bf000080fb0002002000a1ad2100e6
:1024b00002f078003b00370098d2bf0092d2b600fd
:1024c0004040b200370032009252a8009852ae004d
:1024d0009252a900bbd2bf000080fb000000400068
:1024e000612c210060c07800c4f2b70088d2bf0020
:1024f000c452e300160036009012af0013003700fc
:10250000a972ec00a9d2bf000080fb007209200074
:10251000a1ad210002f07800a972ec00a9d2bf00a1
:102520000080fb0012072000a1ad210002f078001e
:10253000a972ec00a9d2bf000080fb00f2072000c6
:10254000a1ad210002f078009012a800150037001c
:102550009012ae0013003700a972ec00a9d2bf00a0
:102560000080fb0072082000a1ad210002f078007d
:10257000a972ec00a9d2bf000080fb001207200066
:10258000a1ad210002f07800a972ec00a9d2bf0031
:102590000080fb0002002000a1ad210002f07800c5
:1025a0009012a9000100200098d2af001140b000a5
:1025b0009272af001140b1002b0032009272a8005d
:1025c00098d2ae009272a900a972ec00a9d2bf0005
:1025d0000080fb00720b2000a1ad210002f078000a
:1025e000a972ec00a9d2bf000080fb0032002000dd
:1025f000a1ad210002f07800a972ec00a9d2bf00c1
:102600008080fb0092d2bf000080fb004300de0010
:10261000a2ad210080707900a972ec00a9d2bf00a0
:102620000080fb0072092000a1ad210002f07800bb
:10263000a972ec00a9d2bf000080fb00c2072000f5
:10264000a1ad210002f07800a972ec00a9d2bf0070
:102650008080fb0092d2bf000080fb004300de00c0
:10266000a2ad210080707900ba12af000501070009
:1026700050c0b300b952b500eb003100b2948000f5
:10268000c3948000d0948000e1948000800f5100ba
:10269000818f5900db0039009df2a800b952e20099
:1026a00035003a00c152e20030003600d09380007d
:1026b0008c12bc00a294880090fd2f00a09488008a
:1026c000a194800070052000808f5000020034002b
:1026d00070052000a0948800a972ec00a9d2bf0068
:1026e0000080fb0072092000a1ad210002f07800fb
:1026f000a972ec00a9d2bf000081fb00a1ad2100ae
:10270000c1d2bf0000f17800a972ec00bbd2bf00bb
:102710000080fb0000004000612c210060c07800b8
:10272000912a2100914078008180fb00a2ad210018
:1027300080707900800220009412b40000067800b6
:102740000c064600608c210060007e00b294800080
:10275000c394800000004100e08049000001be00f9
:1027600032ce880043ce880002003700c6b9ef00a1
:10277000c8b9ef00a200370010c0b300b952e3009f
:1027800018003a00c352e20013003600a972ec00b0
:10279000a9d2bf000080fb00720a2000a1ad210079
:1027a00002f07800a972ec00a9d2bf000081fb0002
:1027b000a1ad2100c3d2bf0000f17800a972ec00e6
:1027c000a9d2bf000080fb0002002000a1ad2100c3
:1027d00002f07800c372ef00cab9ef00ccb9ef0085
:1027e0008700370020c0b300b952e30003003a006d
:1027f000ceb9ef00d0b9ef008100370030c0b30090
:10280000b952e3003a003a00129580002395800007
:1028100020852b00e1f72300bbf7070020928800fa
:1028200031928800a093800030f807000001be00bc
:10283000a0702d0031ba2300b3f707002292800068
:102840003392800052f70700109588002195880088
:10285000bb72ec00129580002395800000002000e0
:1028600001082400a8f7070010f7070000f8070088
:10287000801f7800bbd2bf000081fb000201410035
:10288000612c21004fb17800bbd2bf000080fb005b
:1028900000004000612c21006080780000928800d8
:1028a000bbd2bf008080fb0084d2bf000080fb0051
:1028b000008650000c064600602c210060007e005f
:1028c0004012b50030948800bbd2bf000080fb00ee
:1028d00000004000612c2100608078004400dd0091
:1028e00030638800d2b9ef00d4b9ef00440037005c
:1028f00040c0b300b952e30041003a00bbd2bf0070
:102900000080fb0000004000612c21006080780006
:102910008000780088d2bf000080fb00810f50004b
:10292000030036006c12e200010036006c32ed004c
:10293000f2948000039580003033230031f72300a8
:1029400071f7070020928800319288006093800020
:10295000e6f707000001be00d0cc2c00c1d4230054
:1029600069f70700229280003392800008f7070081
:10297000f094880001958800bd72ec00f09480000e
:1029800001958000baf70700801f7800bdd2bf0014
:102990000081fb0002014100614c21004fb1780031
:1029a000bdd2bf008080fb0082d2bf000080fb0050
:1029b000008650000c064600604c210060007e003e
:1029c000caf707000001be00f09480000195800066
:1029d000eef6070081f70700d0938800bdd2bf0054
:1029e0000080fb0000004000614c21006080780006
:1029f0004500dd0030628800d6b9ef00d8b9ef009d
:102a00002000070099f2ae00060037000621ef0013
:102a10000a21ef000080eb00619c21000900090001
:102a2000801878000400370099f2ae0002003700e9
:102a30000621ef000a21ef00a9d2bf00aa52e3004d
:102a4000090032000188af0007003700aa72ec00cd
:102a5000aad2bf000080fb00a1ad210060c07800b9
:102a60000080fb0020118800120eaa00100ea900a1
:102a70009832af0014cea8009832ae0014cea90050
:102a8000f7fb3700b9f2ef009df2a8005032ef00db
:102a900080928000c200dd00609c21000080400028
:102aa0001000be000001be00d0948000e1948000c0
:102ab000800f5100818f5900090031008092800001
:102ac000c200dd00609c2100008040001000be00bc
:102ad000d0948800e194880050d2bf00b9f2b700ca
:102ae0005032ec0081928000e58f5000e8ff3a0000
:102af000ba12a90000000600b3f2bf0016003200af
:102b000070c0b300b352e30013003e00a972ec00a2
:102b1000a9d2bf000080fb00720b2000a1ad2100f4
:102b200002f07800a972ec00a9d2bf000081fb007e
:102b3000a1ad2100b3d2bf0000f17800a972ec0072
:102b4000a9d2bf000081fb00a1ad2100b4d2bf001b
:102b500000f1780054013700b0c0b300b352e30075
:102b600013003a00a972ec00a9d2bf000080fb005c
:102b7000720b2000a1ad210002f07800a972ec00d8
:102b8000a9d2bf000080fb00b2002000a1ad21004f
:102b900002f07800a972ec00a9d2bf000081fb000e
:102ba000a1ad2100b4d2bf0000f178003e01370092
:102bb000b3d2bf00d1c0b30080cf100016003600e2
:102bc00030c1b300b352e30013003e00a972ec0021
:102bd000a9d2bf000080fb00720b2000a1ad210034
:102be00002f07800a972ec00a9d2bf000081fb00be
:102bf000a1ad2100b3d2bf0000f17800a972ec00b2
:102c0000a9d2bf000081fb00a1ad2100b4d2bf005a
:102c100000f178002401370000c4b300b352e30090
:102c200013003a00a972ec00a9d2bf000080fb009b
:102c3000720b2000a1ad210002f07800a972ec0017
:102c4000a9d2bf000080fb0002042000a1ad21003a
:102c500002f07800a972ec00a9d2bf000081fb004d
:102c6000a1ad2100b4d2bf0000f178000e01370001
:102c700010c4b300b352e30019003a00a972ec008b
:102c8000a9d2bf000080fb00720b2000a1ad210083
:102c900002f07800a972ec00a9d2bf000080fb000e
:102ca00012042000a1ad210002f07800a972ec000e
:102cb000a9d2bf000081fb00a1ad2100b4d2bf00aa
:102cc00000f17800b452e200020036007cb2ef005e
:102cd000010037007c32ef007e32ef00f200370057
:102ce00020c4b300b352e30025003a00a972ec00ff
:102cf000a9d2bf000080fb00720b2000a1ad210013
:102d000002f07800a972ec00a9d2bf000080fb009d
:102d100022042000a1ad210002f07800a972ec008d
:102d2000a9d2bf000081fb00a1ad2100b4d2bf0039
:102d300000f17800b452e20010003a005032ef0087
:102d400081928000e48f500009003e008092800054
:102d5000c200dd00609c210000814000f0ff2f00d8
:102d6000f1ff2f000089be005032ec00f4ff390063
:102d7000ba12a8007e32ef007cb2ef00ca00370022
:102d800060c4b300b352e3001c003a00b4d2bf00e9
:102d90000080fb0000004000209288004452ec00bc
:102da00082f2b700209280001040b00082f2b7009b
:102db000a972ec00a9d2bf000080fb00720b2000ba
:102dc000a1ad210002f07800a972ec00a9d2bf00e9
:102dd0000080fb0062042000a1ad210002f0780019
:102de000a972ec00a9d2bf000081fb00a1ad2100b7
:102df000b4d2bf0000f17800ab00370070c4b3005c
:102e0000b352e3001c003a00b4d2bf000080fb00c4
:102e100000004000209288004452ec0084f2b70089
:102e2000209280001040b00084f2b700a972ec003c
:102e3000a9d2bf000080fb00720b2000a1ad2100d1
:102e400002f07800a972ec00a9d2bf000080fb005c
:102e500072042000a1ad210002f07800a972ec00fc
:102e6000a9d2bf000081fb00a1ad2100b4d2bf00f8
:102e700000f178008c00370080c4b300b352e30047
:102e80000b003a00f0c7b300b452b50005003100a2
:102e9000b4d2bf000080fb004500dd003061880037
:102ea00002003700f0ff2000306188007e0037000c
:102eb00090c4b300b352e30013003a00a972ec00cf
:102ec000a9d2bf000080fb00720b2000a1ad210041
:102ed00002f07800a972ec00a9d2bf000080fb00cc
:102ee00092042000a1ad210002f07800a972ec004c
:102ef000a9d2bf000081fb00a1ad2100b4d2bf0068
:102f000000f1780068003700a0c4b300b352e300ba
:102f100015003a00b4d2bf0088f2b700a972ec00e5
:102f2000a9d2bf000080fb00720b2000a1ad2100e0
:102f300002f07800a972ec00a9d2bf000080fb006b
:102f4000a2042000a1ad210002f07800a972ec00db
:102f5000a9d2bf000081fb00a1ad2100b4d2bf0007
:102f600000f1780050003700d0c4b300b352e30042
:102f70001e003a00b4d2bf0080407800f007200065
:102f800001405000b4f2b700b4d2bf000080fb0093
:102f90004400de00209288004412ec005094880027
:102fa000a972ec00a9d2bf000080fb00720b2000c8
:102fb000a1ad210002f07800a972ec00a9d2bf00f7
:102fc0000080fb00d2042000a1ad210002f07800b7
:102fd000a972ec00a9d2bf000081fb00a1ad2100c5
:102fe000b4d2bf0000f178002f003700e0c4b30076
:102ff000b352e30017003a00b4d2bf000080fb00d8
:103000000020ec0060948800a972ec00a9d2bf00f7
:103010000080fb00720b2000a1ad210002f07800bf
:10302000a972ec00a9d2bf000080fb00e2042000de
:10303000a1ad210002f07800a972ec00a9d2bf0076
:103040000081fb00a1ad2100b4d2bf0000f17800e7
:1030500015003700b0c7b300b352e30012003a00c6
:10306000a972ec00a9d2bf000080fb00720b200007
:10307000a1ad210002f07800a972ec00a9d2bf0036
:103080000080fb00b2072000a1ad210002f0780013
:10309000a972ec00a9d2bf000080fb000200200052
:1030a000a1ad210002f07800b3f2ef0000000600ad
:1030b0007eb2ef0000000600c6b8ef00a0c72500f2
:1030c00040c688005098250050c6880040812500e1
:1030d00060c68800906a250070c6880030542500bc
:1030e00080c68800303e250090c6880090282500c4
:1030f000a0c6880050132500b0c6880060fe2400da
:10310000c0c68800c0e92400d0c6880080d524004d
:10311000e0c6880090c12400f0c68800f0ad24000d
:1031200000c78800a09a240010c78800a087240048
:1031300020c78800f074240030c788009062240003
:1031400040c788008050240050c78800b03e24004b
:1031500060c78800302d240070c78800f01b240051
:1031600080c78800000b240090c7880050fa230015
:10317000a0c78800e0e92300b0c78800c0d92300b9
:10318000c0c78800e0c92300d0c7880040ba230028
:10319000e0c78800e0aa2300f0c78800c09b230096
:1031a00000c88800e08c230010c88800307e23000f
:1031b00020c88800d06f230030c88800a061230099
:1031c00040c88800b053230050c88800f045230051
:1031d00060c888007038230070c88800202b230046
:1031e00080c88800101e230090c88800401123006a
:1031f000a0c8880090042300b0c8880020f82200ee
:10320000c0c88800e0eb2200d0c88800d0df2200d0
:10321000e0c88800f0d32200f0c8880050c822001f
:1032200000c98800d0bc220010c9880080b12200eb
:1032300020c9880070a6220030c98800809b220027
:1032400040c98800c090220050c988002086220012
:1032500060c98800c07b220070c98800807122008c
:1032600080c988006067220090c98800805d2200c4
:10327000a0c98800c0532200b0c98800204a22009b
:10328000c0c98800b0402200d0c988006037220041
:10329000e0c98800402e2200f0c9880040252200a5
:1032a00000ca8800601c220010ca8800b0132200e7
:1032b00020ca8800200b220030ca8800b0022200f9
:1032c00040ca880060fa210050ca880040f22100fc
:1032d00060ca880030ea210070ca880050e22100ec
:1032e00080ca880090da210090ca8800e0d22100cc
:1032f000a0ca880060cb2100b0ca8800f0c32100ba
:10330000c0ca8800b0bc2100d0ca880080b52100a6
:10331000e0ca880080ae2100f0ca880090a7210092
:1033200000cb8800b0a0210010cb8800009a2100bb
:1033300020cb88006093210030cb8800e08c2100f6
:1033400040cb88008086210050cb8800308021004f
:1033500060cb8800007a210070cb8800f0732100d8
:1033600080cb8800f06d210090cb880000682100a0
:10337000a0cb880040622100b0cb8800805c210097
:10338000c0cb8800e0562100d0cb880060512100de
:10339000e0cb8800f04b2100f0cb88009046210064
:1033a00000cc88005041210010cc8800203c210036
:1033b00020cc88001037210030cc8800103221004a
:1033c00040cc8800202d210050cc880040282100ce
:1033d00060cc88008023210070cc8800d01e2100a2
:1033e00080cc8800301a210090cc8800a0152100e4
:1033f000a0cc880020112100b0cc8800c00c210096
:10340000c0cc880070082100d0cc880020042100a6
:10341000e0cc8800f0ff2000f0cc8800d0fb20003a
:1034200000cd8800c0f7200010cd8800d0f3200028
:1034300020cd8800e0ef200030cd880000ec200097
:1034400040cd880030e8200050cd880070e4200096
:1034500060cd8800c0e0200070cd880020dd200015
:1034600080cd880090d9200090cd880010d6200013
:10347000a0cd8800a0d22000b0cd880040cf200091
:10348000c0cd8800e0cb2000d0cd8800a0c82000af
:10349000e0cd880060c52000f0cd880030c220005b
:1034a00000ce880010bf200010ce880000bc200095
:1034b00020ce88000000060000c3b300dafbb7008e
:1034c00020c3b300dbfbb70040c3b300dcfbb70095
:1034d00060c3b300ddfbb70080c3b300defbb70001
:1034e000a0c3b300dffbb700c0c3b300e0fbb7006d
:1034f000e0c3b300e1fbb70000c4b300e2fbb700d8
:1035000020c4b300e3fbb70040c4b300e4fbb70042
:1035100060c4b300e5fbb70080c4b300e6fbb700ae
:10352000a0c4b300e7fbb700c0c4b300e8fbb7001a
:10353000e0c4b300e9fbb70080c3b300eafbb70007
:10354000a0c3b300ebfbb700c0c3b300ecfbb700f4
:10355000e0c3b300edfbb70000c4b300eefbb7005f
:1035600020c4b300effbb70040c4b300f0fbb700ca
:1035700060c4b300f1fbb70080c4b300f2fbb70036
:10358000a0c4b300f3fbb700c0c4b300f4fbb700a2
:10359000e0c4b300f5fbb70000c5b300f6fbb7000d
:1035a00020c5b300f7fbb70040c5b300f8fbb70078
:1035b00060c5b300f9fbb70080c5b300fafbb700e4
:1035c000a0c5b300fbfbb700c0c5b300fcfbb70050
:1035d000e0c5b300fdfbb70000c6b300fefbb700bb
:1035e00020c6b300fffbb70000000600ffff370056
:020000040000fa
:1035f0004012000010000000800000005012000087
:10360000460000008000000096120000100000003c
:1036100080000000a61200002000000080000000d2
:10362000c61200000007000080000000c61900005c
:103630001400000080000000da19000026020000db
:08364000800000000000000002
:00000001FF
